:030000000219FDE5
:03000B000200AA46
:03002B000201606F
:03005B000202E8B6
:030073000202CEB8
:1000800002030406080C10182030406080040608A3
:100090000C10182030406080A0C000070F1F3F0DDB
:1000A0000D04050D050205030302C2AFC0D0C0E078
:1000B000206217E5256002E473E525F4F58A758B67
:1000C00000D262D0E0D0D0D2AF3285268AC262E5BB
:1000D00026F46030758B00D0E0D0D0C295C294C2B7
:1000E00093D2AF32C295C294C293206E0D20660A9D
:1000F0007405D5E0FDE57EF45290758B00D0E0D01C
:10010000D0D2AF32758A00C28DD26201FA01B93005
:100110006805206602D29501B9306805206602D2D2
:100120009401B9306805206602D29301B9D29230A9
:10013000680A2066077403D5E0FDD29501B9D29113
:1001400030680A2066077403D5E0FDD29401B9D265
:100150009030680A2066077403D5E0FDD29301B998
:10016000C2AFC2AD53E6EFC0D0C0E0D2D3D2AFC26F
:10017000CEE52A6007207449152A21C1780079004C
:1001800020742EE580307E01F430E70278FF53DAE8
:10019000CF207E0343DA20307E0343DA10C2D8C278
:1001A00071E580307E01F430E70279FFC3E8997091
:1001B000CB306103752A18207403752A18885FD222
:1001C0007020740DE52B6004152B21D143DA01C298
:1001D000D8207002412FA85F206102C270207436BF
:1001E0007982B70431C3E894F0400374F0F8E8C4AE
:1001F000540F28F87984B703024116C313C3138739
:1002000021200802C313200A06C3C898F841162803
:10021000F8500374FFF88822E52D54066011E53389
:10022000C313C31324062522F52250037522FF7839
:1002300082B6044E852224A824C3E5249564400296
:10024000A864C3E895664002A8668825E56970023F
:100250004180C3E8AA699A5003E8FAE4F9EAC33393
:10026000FBE56BF45B29400D256AF8E56A60021531
:100270006A400B41800AC3E56A9A5002056A78FF1A
:100280008826C3E52594404002D26420CF0AD0E0FE
:10029000D0D043E610D2AD32C2CF053A7801E52A7C
:1002A0006005307402152AC3E55F9401400575624C
:1002B0000041C4756300756C00E5622401F562506D
:1002C000037562FFD0E0D0D043E610D2AD32C2AFAA
:1002D000C0D053E67FC260759100855694855795CE
:1002E000759104D0D0D2AF32C2AF53E6EFC2ADC0E9
:1002F000D0C0E0C0F0D2D3D2AFA8FBA9FCC2D830A6
:100300007102614F53DACF207E0343DA10307E034F
:1003100043DA20D271E580307E01F420E7026126C5
:1003200088278928A17653DACF207E0343DA20304C
:100330007E0343DA10C2D8C271307402A162780021
:10034000E580307E01F430E702A162885FA14A5364
:10035000DACF207E0343DA20307E0343DA10C27105
:10036000206102812853DACF207E0343DA10307EE9
:100370000343DA20C2D8D271885A895BC3E8955802
:10038000F8E99559F97B007E087A00C3E8948CE976
:1003900094005005755E00811A882178A2E6A82194
:1003A0006055C3E894C8E994005008E4D2E4FB7AAD
:1003B0000A61F5C3E89468E994015008E4D2E3FBCC
:1003C0007A0F61F5C3E894D0E994025008E4D2E2D0
:1003D000FB7A1E61F5C3E894A0E994055008E4D2C5
:1003E000E1FB7A3C61F5C3E89498E994085008E48D
:1003F000D2E0FB7A787E00C3E8955CFCE9955DFD70
:1004000030E70AECF42401FCEDF43400FD755E00E5
:10041000C3EC9AED9E5003755E01885C895D855A38
:1004200058855B597802A14AC3E89527F8E99528D1
:10043000F9307C02A12E307B02A12E307A02A12756
:10044000207502814BE9FDE8FC816AE9C313F9E8F4
:1004500013F8307902A127E9C313F9E813F83078CB
:1004600002A127E9C313FDE813FC206126C3EC9425
:0F0470001CED940240028181ED7018C3EC94C81A
:10047F0050120529C3E529940A5002A162755F0045
:10048F00D270A162E529600215297888E6F9740017
:10049F00207F087896B90302789EE624FAFEE434AA
:1004AF0000FFC3EC9EFCED9FFD9208B90310A2085C
:1004BF005007207609D27681CD307602C276A20817
:1004CF005016B9030DECF42401FCEDF43400FD02D9
:1004DF0004E778007900A12EB90315EC33FCED3356
:1004EF00FDC3EC940AFCED9400FD50047C007D00EC
:1004FF00C3EC94FFED9400400678FF7900A12EEC39
:10050F008575F0A4C5F0A2F733F879004003020512
:10051F004A78FF790002054AE9C313F9E813F83066
:10052F007C0EE9600278FFC3E81338F8E43400F971
:10053F00C3E894FFE99400400278FF885FD27020EF
:10054F006102A162741FF4552F4BF52FC274EB702B
:10055F0002D274752A18307403752A0A306102A109
:10056F007620740353DAFE207403752B06D0F0D077
:10057F00E0D0D0D2AD43E6103279010205A679035F
:10058F000205A6790A0205A6791E0205A67964025C
:10059F0005A679C80205A67817E4D5E0FDD8FAD9E3
:1005AF00F6227A147B780205CD7A107B8C0205CD6A
:1005BF007A0D7BB40205CD7A0B7BC80205CD79028B
:1005CF00B27DE4D291D5E0FDD294D5E0FDC294D5B1
:1005DF00E0FDC291D5E0FDD295E576D5E0FDC2955F
:1005EF007496D5E0FDD9D9EAF8D5E0FDD8FBDBCE7E
:1005FF00D29122C37C007D0075F00005F0EA33FA3A
:10060F00EB33FB50F6EB13FBEA13FAC3E9FFE8FEFB
:10061F00E89AF8E99BF95004EFF9EEF8B3EC33FCE4
:10062F00ED33FDD5F0DFEDF9ECF822E889F08A2003
:10063F00D2D4F8A9F07B0030F70B7BFFF42401F83C
:10064F00E9F43400F9E88520F0A4ADF0F8E985204D
:10065F00F0A4AFF0FEED2EF974003FFA7C04C3EA6C
:10066F0013FAE913F9E813F8DCF48BF030F70AE822
:10067F00F42401F8E9F43400F9E889F0C2D4F8A9B8
:10068F00F0227882B604030206ECC3E55F940140C2
:10069F00030206B6852224E4F545F546F547F548ED
:1006AF00F549C26D0206EC7882E6FCD26DE522F5C3
:1006BF0023783879C7AA40AB41C3EB13FBEA13FA8F
:1006CF00EC146013C3EB13FBEA13FAEC141460077A
:1006DF00C3EB13FBEA13FAD1028845894622C3E51F
:1006EF00459523F8E5469400F9500CC3E89480E94A
:1006FF0094FF401602071DC3E8947FE9940050034E
:10070F0002071D787F790002071D788079FF884ADC
:10071F00894B22E54A2547F8E54B3548F9854B20AB
:10072F00E4300701F43549FA30E709C3EA94F040A1
:10073F001502075BC3EA940F500302075B78FF793A
:10074F00FF7A0F02075B780079007AF0C3E52495F2
:10075F0064500AC374019524500B020779E54B20AE
:10076F00E70E020779E54B30E706884789488A4943
:10077F002278A4E6FAC3E54A33F8E54B33F9D13AC8
:10078F00E930E70BC3E89480E994FF4013E1B3C36A
:10079F00E8947FE994005002E1B3787F7900E1B3E8
:1007AF00788079FFE820E715C3E52398F84009C35F
:1007BF00E8940140030207DA78010207DAE8F4242B
:1007CF00012523F840030207DA78FF884C2278A529
:1007DF00E6FAA848A949D13AE930E70CC3E89401F1
:1007EF00E994FF401602080EC3E894FFE994005005
:1007FF000302080E78FF790002080E780179FFE9ED
:10080F0020E715C3E54C98F84009C3E8940140036D
:10081F000208357801020835E8F42401254CF84028
:10082F000302083578FF88242278FFC26420693DCF
:10083F00206A12D264C3E541940A4009C3E52594A6
:10084F00405002C26479A1E76023E541601F74FF45
:10085F008541F0848539F0306A0375F005A4F8C539
:0F086F00F0600278FFC3E895675002A8678866BB
:10087E0022C3E5409440E5419401E566500314011E
:10088E0090046002F566220208982275E89022789C
:10089E0083E6FFE5E820ECF7A8BDA9BE0573C3E526
:1008AE007394084052757300E9FA79A0E76044EA40
:1008BE007007E574601B0208D3C3E895746010E5F9
:1008CE00745006600C140208DF0460F90208DFE5BC
:1008DE0074F574C3946D401B7564C0C394044013C7
:1008EE00756480C39404400B756440C39404400344
:1008FE0075640075BB0622E5642410500274FFF582
:10090E00647982B70402212CC3A864E524985002AE
:10091E00A824C3E895664002A86688258826E57354
:10092E00B4070375BB1022743279A687F0A4C5F004
:10093E00A2F733F8C3E895644002A864882288249D
:10094E00882588268867227540007541F022C2AF3F
:10095E0075C820A8CCA9CDAA3A30CF010A75C824F3
:10096E00D2AFAB3BAC3C883B893CC3E89BF8E99CDF
:10097E00206908F9306702417121CEAD3D8A3DF9FB
:10098E00EA9DFA600478FF79FFAE3EAF3F8B3E8C56
:10099E003FC3EC9FFCC3E99CF542A83BA93CC3E8CE
:1009AE009EF8E99FF9C3E54113FBE54013FAE82AE7
:1009BE00F540E93BF54150067540FF7541FF411882
:1009CE00AA40AB41AC40AD417E047F02C3EB940420
:1009DE0040021E1FC3EB940840021E1FC3ED13FD01
:1009EE00EC13FCDEF7C3EA9CFAEB9DFBEF6009C348
:1009FE00E913F9E813F8DFF7EA28FAEB39FB8A4036
:100A0E008B4150067BFF8B408B41C3EB940250020F
:100A1E00D2673069047F0341437892E6FFC3E5371E
:100A2E00948240110FC3E53794A040010FC3EF9499
:100A3E000640027F057E04E541C4540FF9E541C42A
:100A4E0054F0F8E540C4540F28F8C3E89EFAE99430
:100A5E0000FB4009C3EA9402EB940050047A02E4CE
:100A6E00FB41BDAA40AB41EBC4FEEAC4540F4EFCA1
:100A7E00C3EA9CFAEB9400FBC3E813C313F8EA280D
:100A8E00FAEB3400FB8A408B41C3EB94024002C266
:100A9E00677804EBC4FE7B00EAC4540F4EFAC3EA37
:100AAE0098FA4005C3940250027A027892E6FF301B
:100ABE00600241BD855256855357D26043E680C3CE
:100ACE00E49AF8E49BF93067026157E8FAE9FBD340
:100ADE00E913FDE813FC88528953C3EF9403603881
:100AEE00EF20E00DE82CF8E93DF9ECFAEDFB020BF6
:100AFE0012E828F8E939F9C3E82402F8E93400F9D4
:100B0E007AFE7BFFC3EF9403400E8A548B55884EBA
:100B1E00894F8C508D51618B885489558A4E8B4FDD
:100B2E008C508D51306920C3E53394034019E54252
:100B3E00A2E713F8E555F4240138400B20E70875B9
:100B4E0054FFF42401F555618BE8FAD3E813FC88C1
:100B5E0052C3EF94036020EF20E007E82CF8ECFA84
:100B6E006177E8282402F87AFEC3EF940340088ADE
:100B7E0054884E8C50618B88548A4E8C50E56BC3D2
:100B8E00335002646BF56B3060026195753402D29E
:100B9E006043E680E52D54066026A840A941C3E9CE
:100BAE0013F9E813F8C2AF53E67F759100C3E498CA
:100BBE00F594E499F595759104D26043E680D2AF31
:100BCE0022D265754400752000306B0375204002FB
:100BDE000BEED265754400752040306B0375200016
:100BEE00D2AF7801206722E52D54066002C265C39C
:100BFE00E541940540137802940540087803940566
:100C0E0040027806306902780A206019E5446015C2
:100C1E0030690AC3E53394034003D53406D2AFD20C
:100C2E006C81BF719DD2AF0000C2AF206726E54137
:100C3E00C3FB940F40027B0FEB240530730123306E
:100C4E006A02742820620123F93069027982E58BE9
:100C5E00C39940B50544E59B5440B5200281A930A7
:0F0C6E00690A08C3E8940A40010881172065024B
:100C7D0061EEC26553E67F75910030671075940083
:100C8D007595FE759104D26043E68061EEAE40AF7E
:100C9D0041C3E49EF594E49FF5958190C3E53394AB
:100CAD0002500261EE30650261EED80281BD8117FE
:100CBD00C26C53E67F759100855494855595759159
:100CCD0004854E56854F57D26043E680D2AFE52D51
:100CDD0054066008206A020533020CF9306C0D20B1
:100CED006B0A2065071581158102155F227800308A
:100CFD0064053065027801E53775F007A4F9E5F074
:100D0D0028F5F0E9A2F013A2F113A2F213F537C3FF
:100D1D0094785003753778C3E53795384008D26617
:100D2D00C295C294C293306002A13385505685514D
:100D3D0057D26043E68022207D11C2AF754302D2A7
:100D4D0091C292D2AF759F11020F13C2AF754302BC
:100D5D00D291C290D2AF759F11020F133072432002
:100D6D007D20C2AF75430390013E757E02C293D2C2
:100D7D0090306204D294A187C291D2AF759F0102C7
:100D8D000F13C2AF75430390013E757E02C295D21B
:100D9D0092306204D294A1A7C291D2AF759F210265
:100DAD000F13207D17C2AF754303900119C2933005
:100DBD006202D294D2AF759F01020F13C2AF754379
:100DCD0003900119C295306202D294D2AF759F2162
:100DDD00020F13207D11C2AF754304D292C290D27F
:100DED00AF759F21020F13C2AF754304D290C2920B
:100DFD00D2AF759F01020F13307243207D20C2AF19
:100E0D0075430590012D757E04C294D29130620414
:100E1D00D295C123C292D2AF759F11020F13C2AFEB
:100E2D0075430590014F757E01C294D291306204D5
:100E3D00D293C143C290D2AF759F11020F13207D83
:100E4D0017C2AF75430590010FC294306202D2955F
:100E5D00D2AF759F11020F13C2AF754305900123D9
:100E6D00C2943062EBD293D2AF759F11020F132053
:100E7D007D11C2AF754306D290C291D2AF759F015D
:100E8D00020F13C2AF754306D292C291D2AF759FB6
:100E9D0021020F13307242207D20C2AF75430190A5
:100EAD00014F757E01C295D292306204D293C1BFBB
:100EBD00C290D2AF759F21020F13C2AF754301903F
:100ECD00012D757E04C293D290306204D295C1DF9C
:100EDD00C292D2AF759F01E113207D16C2AF75434B
:100EED0001900123C295306202D293D2AF759F213A
:100EFD00E113C2AF75430190010FC293306202D26C
:100F0D0095D2AF759F01C2662290010D757E00C20C
:100F1D0095C294C293D292D291D290C2622278801D
:100F2D0076090876090876040876FF0876030876B0
:100F3D00FF08760A087601087601087601788C7626
:100F4D00010876FF0876FF0876FF0876FF0876FF22
:100F5D000876030876FF0876FF0876FF08762508E1
:100F6D0076D00876280876500876040876FF08763D
:100F7D000208760008767A0876FF08760108760171
:100F8D00087600087603227887E6FFC2727888E635
:100F9D00C394036008C27DE630E102D27DC27E7843
:100FAD0089E630E102D27EC3EF94026008758E01AE
:100FBD00D273020FC7758E00C273227880E614902B
:100FCD0000809378A4F67881E6149000809378A53C
:100FDD00F67886E61490008D9378A6F6789CE675E3
:100FED0038FF75390CB402067538A075390AB4038B
:100FFD000675388275390578A3E61490009A93F535
:10100D0069120F1622227896E6FA7897E6FB788811
:10101D00E6B40305C3EB940EFB307F047A007BFF2F
:10102D00C3EB9AFCC3948250027C827575000575E2
:10103D00EC8575F0A4C3E5F0947D40F222D27F11CA
:10104D00131205977A007B007C1012058DE55F2A3F
:10105D00FA74003BFBDCF37C04C3EB13FBEA13FADD
:0D106D00DCF7FEC27F111322E5EF20E60341
:10107A007520000520903FFFE520146006901DFFB3
:10108A001460009304600375EF1253D9BF7581C0D1
:10109A0043FF8012058875EF0243B203E5B32404C7
:1010AA0020E70DF521E5E320E0068521B343E301BE
:1010BA00120F167580FF75A40075F19075D47F75AF
:1010CA00908775A5BF75F2BF75D50075A60175E243
:1010DA0041E4F8F6D8FD756B01120F2B1215A178B1
:1010EA00988676753001C2AF1205A11205B11205B4
:1010FA00971205B81205971205BF120597C2AF7865
:10110A00FA79FA308707D9FBD8F7021C00120F9434
:10111A00120FC81112111378988676120F16758855
:10112A005075891275C82475910475D84075A8221E
:10113A0075B80275E690759B80759D0075D10E7520
:10114A00BC5875BB0675BA1175E880120588D2AF0E
:10115A0012089553DACF207E0343DA20307E034308
:10116A00DA1043DA01C2D8C2711205A1D2617B0337
:10117A007A0CE55E70077A0CDB03021107120597F9
:10118A00207003021107C270E55FC3940240E1E5D3
:10119A002F541F856160F561B560D5DAD5C26153F8
:1011AA00DACF207E0343DA20307E0343DA10C2D836
:1011BA00C27178A2E67008D274E52F54E0F52FC206
:1011CA007575290012059C307409C3E529940A40F3
:1011DA0002D27512058D78023074027800C3E55F79
:1011EA009840F0C2AF1205B11205B11205B1D2AFE3
:1011FA001205A1754D007888E6B4030241DE120596
:10120A008D788CE6C3940150030212DEE530C39454
:10121A000150030212DE207435C3E55F94FF5003C8
:10122A000212DEC2AF1205C6D2AF12059CC3E55F39
:10123A00940150EFC2AF1205B11205921205B1D254
:10124A00AF12059CC3E55F94FF40E90217497F028C
:10125A00D27F111312059CC2AFC27F1113AE5FC3B6
:10126A00E55F947FD2AF4076120588C2AF1205C6F9
:10127A00D2AFDFDC114AC3EE94057897F61205A1C6
:10128A001215E31216CC7F0AD27F111312059CC2E3
:10129A00AFC27F1113AE5FC3E55F947FD2AF50E652
:1012AA00120588C2AF1205B11205921205B1D2AF6A
:1012BA00DFD6114AEE24057896F61205A11215E337
:1012CA001216FB12059C1113C3E55F94FF500241ED
:1012DA0020021749C3E55F954D4003855F4D12050E
:1012EA009C78017988E7B403027805C3E55F9840E2
:1012FA00024100C2AF1205C61205C61205C6D2AF18
:10130A001205A1753000E4F531F5320531E531F405
:10131A0070390532789AE6781914601278321460B6
:10132A000D787D14600878FA146003753200C3E5FD
:10133A003298401715327531B478998676C2AF1251
:10134A0005C6D2AF7898867612059C120592E52AD0
:10135A007005307402210778012074027806C3E50B
:10136A005F9840A77888E6C39403600312059CE55A
:10137A002A7003021107C2AF120F16E4F522F523F1
:10138A00F524F525F526F56AD2AF7885E6C333F557
:10139A0068E4F545F546F547F548F549F573F52C42
:1013AA00F52DF53775730875BB1012058812089963
:1013BA00E5E820ECFBA8BDA9BEE97001F888741223
:1013CA00089D75730875BB107887E6FE7602120FC2
:1013DA00947887EEF6C2AF7564FF120935852264E8
:1013EA00852265852266D2AF75220175240175258D
:1013FA000175260185636C756D017888E6B403076B
:10140A00C27D307602D27DD268D269753300120E5F
:10141A007C120EA112095512095C12095512095CB7
:10142A0012095502143DC2AF120F94D2AF75730060
:10143A0075BB06120BE0120691120CFA120D441239
:10144A00095C120BCF306D031206ED2067031208F8
:10145A003830670312087F120CFA120D6912095C00
:0F146A00120BE0306D03120722120CFA120DE084
:1014790012095C120BCF306D03120780120CFA129D
:101489000E0512095C120BE0306D031207DD120C18
:10149900FA120E7C12095C120899120BCF120CFA7F
:1014A900120EA112089D12095C306935206B328534
:1014B900676485676585636C756D0179187A0CC3F6
:1014C900E53399400FC269D26A8A358567648567B1
:1014D900660214EAC3E55F9401400302143D021554
:1014E90067306A1B206B18E535147004C26A8130B5
:1014F900F535C3E55F9401400302143D0215677594
:101509003600C3E56278FA985054307404E52A60CD
:101519004D7888E6B40317207D05207607A137307A
:101529007602A137206B07D26B856764817C78F0DE
:10153900306B058567647820C3E541985002813D89
:10154900306B1BC26BC27D307602D27DD26A753593
:1015590012856764813D0536E55F6002A16A7536CB
:1015690000C2AF120F167887E6FE7602120F947842
:1015790087EEF6E4F522F523F524F525F526F56839
:10158900C268D2AF120588120F16307409C3E53646
:101599009405400221076110901A0D782012162532
:1015A900E520B4550CA3121625E520B4AA030215AB
:1015B900C3120F2B1215E30215E2901A0378807BF0
:1015C9000A121625A308DBF9901A0F788C7B1812DA
:1015D9001625A308DBF9901A2722C2AF1216641246
:1015E900163E901A00740E12162AA3740412162AB3
:1015F900A3741412162A901A0378807B0A121629EA
:10160900A308DBF9901A0F788C7B18121629A30806
:10161900DBF9121677121655901A2722E493F6224F
:10162900E6438F01538FFD75EF0275B7A575B7F1C5
:10163900F0538FFE22438F02438F0175EF0275B776
:10164900A575B7F1901A0DF0538FFC22901A0D74FD
:1016590055D12A901A0E74AAD12A227A3079D078D3
:1016690020901A40D125E520F709A3DAF7227A302C
:1016790079D0901A40E7D12A09A3DAF922AB77A8E1
:1016890078BB01027980BB02027981BB03027982AE
:10169900BB04027984BB05027986BB06027992BB39
:1016A90007027987BB080279A3BB0902799CBB0AA7
:1016B900027988BB0B027989E8F7227C051205A11A
:1016C900DCFB22C2AF1205B11205B81205BF120523
:1016D900C61205921205B11205B81205BF1205C648
:1016E9001205921205B11205B81205BF1205C6D22C
:1016F900AF22C2AF1205C61205BF1205B81205B155
:101709001205921205C61205BF1205B81205B112CB
:1017190005921205C61205BF1205B81205B1D2AF5E
:1017290022AE77AF78C2AF1205B11205B11205B179
:10173900120592DEF21205C6120592DFF8D2AF2227
:10174900D1CCD1C4D1C4757701757801757900F10F
:101759002A7C05AD5F1205A1C3ED955F70F5C3E560
:101769005F9401400AC3E55F94FF4032021785D1B7
:1017790086B1E3D1CCC2AF75EF12D1C4DCD50579FE
:10178900C3E5799403500280C6D1C40578E577147E
:1017990090009F93F808C3E57898500280AED1C4B1
:1017A900D1C40577C3E577940C5002809C120F2BA6
:0917B900B1E3C2AF75EF12D1C417
:0319FD0002107560
:101A00000E0414090904FF03FF0A01010155AA018C
:101A1000FFFFFFFFFF03FFFFFF25D0285004FF0259
:081A2000007AFF01010003FF41
:101A400023585031384123202020202020202020DE
:101A500023424C48454C4923463333302320202031
:101A60002020202020202020202020202020202076
:101C0000C2AFC2D353D9BF7581C043B20343FF8073
:101C1000752438752503B1C975EF0275E24043F1AB
:101C20008053A47F75D400D2877DFA780379E67C4F
:101C300010752200752300901DD67B0675249875BB
:101C400025013087028142208708D8FBD9F9DCF7CB
:101C500081B4308708D8FBD9F9DCF781B4B189E4C5
:101C600093A3C39A6004DDC381B4DBDBB17B600264
:101C7000812B7B08E493FAA3B15CDBF87A30B15C8A
:101C8000752200752300B17BEAFCEBFDC3ED94FEE9
:101C9000400EB17B8A278B28ED30E0048A828B834B
:101CA000B17B7AC270D8C3ED94FE601350CEBD00F4
:101CB00025EC60097520007521FF0200008100A855
:101CC00027A9280809D804D90281D3B17FEA89AAB3
:101CD000F281C50D81A0C3ED94035049EDA2E092BD
:101CE000007AC5C3E5829400E583941C50902000DF
:101CF00010438F02438F0175B7A575B7F1F030001F
:101D00001FA827A9280809438F01538FFDD804D99C
:101D100002A12089AAE275B7A575B7F1F0A3A10DBC
:101D2000538FFC817C7AC1BD030CE493A3FAB140CC
:101D3000DCF8B138817C817EAA22AB23B15CEBFA5E
:101D4000EA6222752608C3E52313F523E52213F57D
:101D50002250066323A0632201D526EAB1C9B1C986
:101D600075260AEAF4200102D287300102C287B147
:101D7000C9C3134002C201D526EB22B17FEAFB2082
:101D80008702A17F308702A184752608AE24AF2583
:101D9000C3EF13FFEE13FEB1CDB1C9C3EA13308711
:101DA000024480FA30E703632201C3E52313F523DD
:101DB000E52213F52250066323A0632201D526D91C
:101DC000E52265236523F52222AE24AF250E0FDE22
:101DD000FEDFFCD20122424C48656C693437316326
:041DE000F3300601D5
:00000001FF
